:020000040800F2
:10500000381A0020D550000885820008757A0008FB
:105010000000000000000000000000000000000090
:10502000000000000000000000000000F18C0008FB
:105030000000000000000000FD880008ED8D000861
:10504000E7500008E7500008E7500008E750000864
:10505000E7500008295B0008E7500008E750000807
:1050600000000000E7500008515A0008E75000080F
:10507000E7500008E17E000800000000E75000084B
:1050800000000000E75000080000000000000000E1
:10509000E750000800000000E7500008E750000853
:1050A000E7500008E7500008E75000086595000841
:1050B000E7500008E7500008000000000000000072
:1050C0000348854600F060FC0048004775A30008CF
:1050D000381A00200448804704480047FEE7FEE7EE
:1050E000FEE7FEE7FEE7FEE7898E0008C1500008F4
:1050F00030B50B46014600202022012409E00D4670
:10510000D5409D4205D31D469540491B25469540F7
:1051100040191546521E002DF1DC30BDF0B51FB40C
:105120000646002082B005464024019100901BE015
:10513000019922460F46304600F04EFB049A059B2B
:10514000801A994110D310461946224600F034FBCC
:10515000361A8F410197224601200021009F00F05E
:105160002BFB38184D4100902046641E0028DFDCE0
:10517000019B00982946324607B0F0BD03460B4319
:105180009B0703D009E008C9121F08C0042AFAD2FD
:1051900003E00B780370401C491C521EF9D2704783
:1051A000D2B201E00270401C491EFBD270470022BF
:1051B000F6E710B513460A4604461946FFF7F0FF16
:1051C000204610BD30B504460020034600E05B1CBD
:1051D000934203D2E05CCD5C401BF8D030BDF8B503
:1051E00002464A40D40F42004B0052085B089A42E4
:1051F00002D20246084611464A0023D0C30D4A0097
:10520000DDB2120EAD1A202D35DA49020126490A07
:10521000F6058A19002C00D0524220214F1B11465E
:10522000B9402A411018C20D9A4221D0002C17D043
:10523000012D08DCDA05801AD20F8019D207DBB203
:1052400000F0F6FAF8BDDA05801A012340001B06CB
:10525000C01880185A428018CA0F1043490007E04E
:105260004908C2071143DA05801A801940088018DE
:1052700000F0D6FAF8BD61000122511A001BF7E7D1
:105280000122D2075140AAE70122D2075040A6E7E7
:1052900070B502464A40D50F40004A00ED0740086D
:1052A0005208002814D0002A12D0C40DD30D410298
:1052B0000120C0055202490A520AE41A09181218BC
:1052C0007D34914201D3641C00E04900002C01DAD6
:1052D000002070BD0023914201D3891A0343400886
:1052E00049000028F7D100290AD0914202D10121BA
:1052F000C90705E0914201D2012101E00121C94322
:10530000E005C018401900F08BFA70BDF0B50746F3
:105310000846584087B0C00F049048000E46590018
:1053200040084908BC1A884105D2384631461E4615
:1053300017460B4602465800400810434CD0300D2B
:10534000039040055900400D490D0590401A029008
:10535000402872DA18030121000B09050843019067
:1053600004980092002805D00199524200208841FB
:1053700000920190029840210A1A0199009800F0C9
:105380001BFA05460C466B4607CB00F036FAC019EF
:105390007141039A0E0D0023D71756401A467A40E2
:1053A000164344D0049A002A2DD0029A012A039A67
:1053B00015DC1205C01A914101263605001C714109
:1053C000D20F059ED2070093019202962A462346E9
:1053D00000F074FA07B0F0BD38463146FAE716051A
:1053E000224A0F46B218C01AB74101210905001C14
:1053F0004F4100187F41114618187941E20F1043C0
:105400006D19644113E0E2076D0815436408C20793
:105410001443039A01261205C01A91413605001C57
:105420007141CE07400830434908C01851412A460F
:10543000234600F036FACDE7FFE70498012240004A
:10544000C117121A00238B4104983146C417381A29
:10545000A141EEE730B40124E407634030BC55E7D6
:1054600030B40124E407614030BC4FE70000E0FFA6
:10547000F0B51FB488B00B990998002448400999E9
:10548000C00F490049080991C0070B9900904900D5
:1054900049080B9109990898A64608431CD00B9916
:1054A0000A98084318D0099801244000420D48008A
:1054B000410D099824050003000B204309900B9827
:1054C0000003000B20430B9050181C494018002289
:1054D00001901446104605E0002001460DB0F0BDD5
:1054E000032801DA034600E003239C46C11A0AAEF2
:1054F0000AE05F0008ADED5B4F00F75B7D430027DE
:10550000AA187C41491C5B1E6145F2DD410004ABD9
:105510005A522104120C0A43240C401C0828DFDBD9
:10552000019802900099704601910090059B049AA1
:105530000799069800F0C2F9D0E700000DFCFFFFC4
:10554000F0B50C465C4085B0E40FE40703944C00D2
:1055500000266408590094464908024602962243F0
:1055600021D062460A431ED06200570D4A000E0346
:105570002303550D012402462C492405781B1B0BDF
:10558000360B401823432643614600901C46501AB0
:10559000B44103D30098401C009002E09218009898
:1055A0005B41002803DA0020014605B0F0BD002071
:1055B000012109050746864611E064461D46141B75
:1055C000B54106D36546521BB341744607430C43AD
:1055D000A646CD0740084908284392185B41054676
:1055E0000D43EAD11046184313D060461946504087
:1055F0007140084306D06046101AB34106D201221A
:10560000002306E000220123DB0702E00122D2434F
:105610005310009874460105381C6141029C039D9B
:105620000019694100F03DF9BFE70000FD030000EB
:10563000C217C10F504010B54018CA079623002169
:1056400000F0F6F810BD10B500229623114600F0C8
:10565000EFF810BD0EB5C217C10F5040CA07401871
:105660000021054B0293019200910A460B4600F07F
:1056700025F903B000BD0000330400000EB5054954
:105680000291002100910A460B46019100F016F9A3
:1056900003B000BD33040000410040020122400A73
:1056A000D205090E80187F2901DA0020704796295B
:1056B00003DC9622511AC8407047963988407047DB
:1056C00070B5CD0F4A0009030123090B1B051943CF
:1056D0000B4BED070024520D9A4201DA002070BDF9
:1056E000074B34339A4203DC9A1A00F075F802E053
:1056F0000449511888402C43F1D0404270BD00004D
:10570000FF030000CDFBFFFF4A0009030123090B43
:105710001B051943094B10B5520D9A4201DA0020BE
:1057200010BD064B34339A4203DC9A1A00F054F849
:1057300010BD03495118884010BD0000FF03000050
:10574000CDFBFFFFC20FD207400040080BD0C10DB8
:105750000723DB01C91840020905400A1143C208AA
:10576000400711437047002001467047CB0FDB070D
:10577000490010B5490802460A4307D00A0D07241C
:105780000903E401090B121B002A01DC002010BDF3
:10579000C900440F0C43C100E018D205801800F086
:1057A0003FF810BD0122D207002800DB101A0029A3
:1057B00000DB511A8142704710B5202A04DB0146F4
:1057C000203A9140002010BD914020239C1A0346AE
:1057D000E3401943904010BD10B5202A04DB084671
:1057E000203AD040002110BD0B46D340D0402024A9
:1057F000A21A91400843194610BD10B5202A06DBB5
:10580000CB170846203A1041C1170B4306E00B4660
:105810001341D0402024A21A91400843194610BDDC
:10582000002904DA401C490001D1400840007047BB
:1058300070B40024050C05D11024000402D1002905
:1058400021D01124050E01D100020834050F01D129
:105850000001241D850F01D18000A41C002801DB5C
:105860004000641C002908D020252E1B0D46F54061
:10587000A14000D001212943084301061B1B000A57
:10588000DB1D02D5002070BC7047DB05181880189E
:105890000029F8DA401C4900F5D170BC40084000EE
:1058A000704710B5002B08DA0024401C61419218A3
:1058B0005B411A4301D14008400010BDF0B51FB450
:1058C00082B005460C0003D0084603F009FF02E051
:1058D00003F006FF20300246009021462846FFF7DD
:1058E0006BFF049B059A04460F4618431143084377
:1058F00014D0184610431BD0009840210A1A1846AD
:105900000599FFF769FF05460E46009A0599049828
:10591000FFF752FF084305D0012004E02046394636
:1059200007B0F0BD0020C11705430E432C43374399
:1059300000990E986305401A7905E40A00220C4389
:10594000FD0A0A3002D500200146E9E701051019D9
:1059500069410C9C0D9D00196941FFF7A2FFDFE72B
:1059600010B5002904DB0124E40740428C412146A4
:10597000002B04DB1C460123DB075242A341994262
:1059800000D1904210BD0000064C0125064E05E0F6
:10599000E36807CC2B430C3C98471034B442F7D350
:1059A000FFF792FBD4A60008F4A6000838B5044619
:1059B000064805490068FFF79BFB604300E0401E76
:1059C00000900028FBD138BD40420F00EC000020C1
:1059D000F8B50446006881688907890F012902D15A
:1059E0000168C90722D18168114A1026114001259A
:1059F00000290ED18168294381600120FFF7D6FF7D
:105A000000F0A8FF07460CE000F0A4FFC01B0A2826
:105A100007D9606D30436065A06D2843A065012003
:105A2000F8BD20680068C043C007EDD10020F8BD74
:105A30001700008010B500231A4603E0845CE318C9
:105A40009BB2521C8A42F9D3D84380B210BD0000E9
:105A500010B5034800F03EFD024800F03BFD10BDCC
:105A6000D81500209015002030B5446C1C252C4022
:105A70000125A540046C6560046863608368102B91
:105A8000036803D099600068C26030BD9A60006806
:105A9000C16030BD1449012048720A4602205E32BE
:105AA000507203203C3A507204200E3A50720F4854
:105AB0000D4B0078087022310870203108770C49AE
:105AC0005A1C0878587149789971233318715971A3
:105AD000203318775977107551751A461E32107594
:105AE000517510765176704720110020BE000020BD
:105AF000D800002010B503F0D3F8202003F06CF993
:105B0000012004F09DF9002003F066F9044804F038
:105B10003BF8044804F0DEFA002004F013FB10BD4B
:105B2000A80000208380000070B505200121000737
:105B300000F000FF00240D4D002800D02C60022151
:105B40000B4800F0F7FE002808D10A482C600088B6
:105B50000A2148430849088003F016FD012000F09F
:105B600021FE022000F01EFE70BD0000E4000020B7
:105B700000040050CC000020D60000207047000038
:105B800010B5084900224A6107494B684C15234368
:105B90004B604B68082423434B60C009C00102607E
:105BA00010BD000020160020002002407FB5002517
:105BB0000C460646039500F0C5FDE009029003A9D6
:105BC00001960095684600F055FD002804D000F0CD
:105BD0008DFD002004B070BD00F088FD0120F9E7C4
:105BE00010B5002302E0C45CCC545B1C9342FAD392
:105BF00010BD000010B5214A00219069C30520485E
:105C000004D54169022319434161911593699B05AC
:105C100005D5436901242343436163021943936912
:105C20005B0505D54369082423434361E301194318
:105C300093691B0505D5436904242343436163022B
:105C4000194393699B0405D5436910242343436199
:105C50006302194393699B0304D5446920231C43C1
:105C6000446119439369DB0305D543694024234309
:105C70004361A0020143916110BD00000020024079
:105C80002016002070B5054600F064FE0646184C4C
:105C90000AE0681C08D0002D04D000F05BFE801BD9
:105CA000A84201D9032070BDA069C007F1D1A06945
:105CB000800701D50220A061A069C00511D4A069A8
:105CC00080050ED4A06940050BD4A069000508D456
:105CD000A069800405D4A069800302D4A069C00330
:105CE00003D5FFF787FF012070BD002070BD0000C5
:105CF00000200240F8B51746002605460C4600F085
:105D000021FD09E029460220226800F0FDFC002860
:105D100004D1241D2D1D361DBE42F3D300F0E6FC38
:105D2000BE4201D20020F8BD0120F8BD10B50849DF
:105D300002460020054B497905E044001C5B944273
:105D400003D0401CC0B28842F7D310BD48120020D7
:105D50004800002010B500F0F2FD10BD10B5094854
:105D600000F09AFF80B2FFF789FC074A074BFFF764
:105D70007FFB0022064BFFF7E3FBFFF7C5FC80B279
:105D800010BD000088140020F853E3A59B843E401A
:105D900000408F40F8B53F4C3D48217F0175617F41
:105DA00041753D490A78027649784176384905209F
:105DB000133148720A2004F07DF9002004F094F9B0
:105DC0003349002213310C2004F05EFA00210C202C
:105DD00004F06CFA022004F0BDF9304D00210F20D0
:105DE00004F0E8F82842E062F8D0E06A411C40D0B4
:105DF0002B4E2C4F40043ED58122D20100210F2092
:105E000004F017FA0021102004F0D4F841062048CD
:105E1000490E0022633004F003F91D4D6335687AA2
:105E2000052825D102221C49681DFFF7CBF900285F
:105E30001ED1A87A607117480422691C4030FFF710
:105E40009DF9206C00F034F86083607929464200A7
:105E50000B3108465930FFF791F913483188808893
:105E6000FFF746F93888414310480180022020702E
:105E7000F8BD02F02BFA608B31880546FFF738F940
:105E80003888414309486D1E01806583F8BD0000D4
:105E90008111002048000020D800002000D02724D5
:105EA000C8000020C6000020200D0020C4000020F3
:105EB00010B504460E4800F0EFFE0E49C006C00EB5
:105EC000098805E02246C240D2070FD0401CC0B26C
:105ED0008842F7D3012005E02246C240D20705D010
:105EE000401CC0B28842F7D3491EC8B210BD0000A2
:105EF00088140020C800002010B5084800F096FA69
:105F00000A21064800F032FA044800F01DF9800525
:105F100003D5024800F01AF980B210BD2C140020FD
:105F2000F8B52F4D00220121284600F00CFDFFF7A7
:105F3000E3FFFFF788FB2B4E3146FFF7A9F92A4C08
:105F40000122A0601146284600F0FDFC2749A06808
:105F5000002588423EDB2078254F002815D025708B
:105F6000FFF7CAFFFFF76FFB3146FFF791F9A0601B
:105F7000FFF7E8FB00223B46FFF76CFA00221D4BBF
:105F8000FFF776FAFFF7F2FB6060A068FFF7DAFB35
:105F900000223B46FFF75EFA174A184BFFF768FAF4
:105FA00006460F466068FFF7CDFB134A144B52427A
:105FB000FFF75EFA32463B46FFF7A8F9FFF7D6FB3C
:105FC00010496060884201DD616004E0FF21C9057D
:105FD000C84200D365606068FFF75EFBC0B2F8BDE1
:105FE0000004005000401B442400002000006040DA
:105FF00000000C4000E064403333333333B33040AF
:10600000CCCCEC3F0000C842F8B50546044640350C
:10601000287C0026012808D0012028742068816887
:106020008907890F01290ED101E00220F8BD01681E
:10603000C90708D0606D2021084360650126002053
:1060400028743046F8BD616DFF220132914302226F
:1060500011436165C1688907890F0091C16889088A
:106060008900C1602068816892071143816000F057
:1060700071FC07460EE000F06DFCC01B0A2809D930
:10608000606D022188431021084360650020287458
:106090000120F8BD206880680028ECDB2068C1681A
:1060A000009A1143C160606D80088000401C6065EB
:1060B000C5E70000F8B506460D464036317C01299B
:1060C0000DD00121317401688A68520709D5416DEC
:1060D000202211434165002030740120F8BD0220C8
:1060E000F8BD174B6A68D80547109A42154C8A6A62
:1060F0002B6812D05B035B0B1A438A622968490341
:1061000005D5A1680143A1600A20FFF74FFC28686C
:10611000800312D5A06838430EE05B035B0B9A4303
:106120008A622968490302D5A1688143A160286871
:10613000800302D5A068B843A06000203074F8BD89
:106140000110000000270140406D70470068006C9E
:106150007047000070B5040006D0606D264600252B
:106160004036002802D006E0012070BDA5653574D8
:10617000204600F0D3F8606DC00603D4216888681B
:10618000400705D5606D1021084360653574EBE765
:10619000606DFF22013290430222104360658868DF
:1061A0008207920F5B48012A02D10A68D2072BD1DD
:1061B000032362689B079A4205D05B429A4202D051
:1061C0005B009A4209D10A69920092080A6121682B
:1061D0000A6963681A430A610CE00A69920092082E
:1061E0000A6181680F22920491438160816862682C
:1061F000114381602168CA6818239A43CA602168E4
:10620000CA68A3681A43CA60816801225206914392
:1062100081608168A28E5206114381602068816886
:10622000C90004D4816801221207114381602068EB
:10623000C168394A1140C1602069E168022825D04F
:1062400000200143204620300278037B52035B008C
:106250001A431143226B1143A26992031143E2696D
:10626000D20311432268D3681943D160616A0A4698
:10627000FF3AC23A05D0A26A11432268D368194393
:10628000D16042780121012A02D00BE00420D8E736
:106290000078002823D0606D202210436065A06D37
:1062A0000843A065E06B012820681FD00169C90779
:1062B00003D0016949084900016120684169C908A2
:1062C000C900416120684169A26B11434161A56524
:1062D000606D80088000401C6065002070BD2068F3
:1062E000C26801231B041A43C260DBE70269FF2373
:1062F0009B009A43026120680269236CA66C1A43D2
:10630000636C33431A430261206802690A430261E5
:10631000D3E70000002701401902FEFF10B586B048
:10632000044614216846FEF742FF0E492068884261
:1063300016D10D48416B421511434163C16A0122D8
:106340001143C162C06A6946104005900220009066
:1063500003200190002002900520000700F02EFA93
:1063600006B010BD0024014000100240F8B50446FC
:106370004069254640350E4608280BD02068C06885
:10638000C00709D0606D2021084360650020287493
:106390000120F8BD082700E00C2700F0DBFA009090
:1063A00011E0701C0FD0002E05D000F0D3FA009938
:1063B000401AB04207D9606D04210843606500208F
:1063C00028740320F8BD206800683842E9D0606D69
:1063D00001214902084360652068C16809058A0FE8
:1063E0000C21002A1BD12022125D002A17D102683D
:1063F000120714D5826853070122002B08DB43687B
:106400008B434360606D130298431043606506E060
:10641000606D202318436065A06D1043A065A069DE
:10642000002801D1206801600020F8BD70B5044645
:10643000216800208968490721D425464035297CF8
:1064400001291CD001212974E169012904D02046C9
:10645000FFF7BEFA002811D1616D0A4A1140FF22F0
:106460000132114361650021A165297422681C2154
:10647000116021688A6804231A438A6070BD022073
:1064800070BD0000FEF1FFFF70B500240146203111
:106490004A79022A03D00421C163012418E002686A
:1064A00013680E25AB431360026813685B085B003A
:1064B0001360436C1C221340012215469D40036C5F
:1064C0005D604A7100220A71816B002900D0884703
:1064D000204670BDF0B4016C0D6801680C68466C14
:1064E0001C2304221E401746B7402F420ED06707D8
:1064F0000CD50C68A40602D40C6894430C60416C63
:1065000019408A40016C4A60016B1AE00227B740CB
:1065100002462F402032002F17D0A70715D50C6850
:10652000A40605D40C680A25AC430C600121517106
:10653000446C02211C40036CA14059600021117180
:10654000C16A002918D0F0BC08470827B7402F427D
:1065500012D0240710D50C680E25AC430C60446C97
:1065600001211C400B46A340046C6360C163517160
:1065700000211171416BE4E7F0BC704770B5040075
:106580003CD01F48256814212818FEF7B1FD800073
:1065900060641C482064022120462030024641717C
:1065A00029681948E3680140A068666918432369AF
:1065B00033431843A3691843E3691843236A184314
:1065C000084328600121A0688903884210D00D4843
:1065D0008030836A656C1C210D400F26AE40B343AA
:1065E0008362656C63680D40816AAB400B438362D4
:1065F0000020E06301215171107170BD012070BD58
:10660000F8FFFDBF000002400F80FFFFF8B5044611
:106610008C46203001790025012909D00126067118
:1066200041790027012905D0077102252846F8BDC8
:106630000220F8BD02214171E76320680168490822
:106640004900016061462046FFF70EFA206B0028E2
:106650002068016801D00E2205E004229143016008
:10666000206801680A2211430160206801683143F3
:106670000160DBE7F8B51A4E0546307C0F4601286D
:1066800007D0012030741748FFF7FCFA010002D050
:1066900021E00220F8BD0020C04338606C6814E09F
:1066A0002046FFF76DFA0F48FFF7ECFA01460E4857
:1066B000426808239A434260426843159A43426005
:1066C000002901D03C6006E08034A8686A68C001F7
:1066D0008018A042E4D8002030740846F8BD0000BD
:1066E0002016002050C300000020024005484168E9
:1066F00002221143416041680122114341600020A0
:106700007047000000200240F8B50C4C1646207C73
:106710000F46012808D0012020740948FFF7B2FA7B
:106720000025002802D006E00220F8BD65613E6029
:106730000348FFF7A7FA2574F8BD000020160020D3
:1067400050C3000011484168C9070BD0EFF3108116
:1067500072B60F4AC2600F4AC26081F31088416866
:10676000C9070ED1416889070DD5EFF3108172B6C4
:10677000094A0261094A026181F310884068800772
:1067800001D5012070470020704700000020024022
:10679000EFCDAB8905040302BFAE9D8C1615141313
:1067A0007047000010B504494A69024202D04861AE
:1067B000FFF7F6FF10BD000000040140F8B500230C
:1067C0000124A2E027469F403A4070D04D68022D38
:1067D00001D0122D14D1DD08AD002D1800952D6AC1
:1067E0005E07AC46F50E0F26AE46AE406546B54395
:1067F000AC460E697546AE4065462E43009D2E623E
:106800004D68012D05D0022D03D0112D01D0122D80
:1068100016D185680326AC465D00AE46AE4065469F
:10682000B543AC46CE687546AE4065462E4386609D
:1068300046680D79BE43ED06ED0F9D40354345603A
:1068400006685F000325BD40AE46AE430D79B446F1
:10685000AE07B60FBE4065462E430660C668754655
:10686000AE438D68BD403543C5604D68ED004BD5E6
:10687000294D6E6B26436E639E08284DB600751930
:10688000AC46AD689E07360F0F27B740BD430527BE
:106890003F07B84201D1002715E0214FB84201D18E
:1068A000012710E01F4FB84202D102270BE02BE076
:1068B0001D4FB84201D1032705E01C4FB84201D15A
:1068C000052700E00627B7402F436546AF60184D07
:1068D0002E684F689643FF0300D516432E606E68FE
:1068E0004F689643BF0300D516436E60AE684F688D
:1068F0009643FF0200D51643AE60EE684F6896439C
:10690000BF0200D51643EE605B1C0A681546DD40E9
:1069100000D057E7F8BD0000001002400000014021
:106920000004005000080050000C0050001C0050F3
:10693000000401400069084000D00120704742690E
:106940004A4042617047002A01D0816170478162EC
:10695000704700000148006870470000E800002010
:1069600002480168491C016070470000E8000020EF
:1069700010B50848002401684022114301602046F8
:1069800000F00AF8002801D0012401E000F0B0F97D
:10699000204610BD0020024070B5054609487D2103
:1069A0000024C9000068FEF7A3FB00F045FE0028A4
:1069B00001D0012404E000222946501E00F0B8F95D
:1069C000204670BDEC00002070477047F8B52C4C95
:1069D00001266078401C6070E670208B401C20838C
:1069E000208902F0C3F9274DE888FEF72CFE2649DE
:1069F000FEF74EFC254F3968FEF7F1FB38600221A7
:106A00002348FFF797FF002809D0002020621F4885
:106A10002049076820488F4212DD067012E0E8889E
:106A2000FEF711FE1849FEF733FC216AFEF7D7FB8B
:106A30001A4920628842EADB1A491948C860E6E729
:106A400000210170688F401EFEF7F2FD3946FEF707
:106A5000A9FE06D82079002803D01348C179314314
:106A6000C171688FFEF7EFFD08490968FEF79AFECD
:106A700004D22079002801D003F000FDF8BD000009
:106A8000BC000020200D002000007A44E40000201B
:106A900000040050000040404E0000200000A040D4
:106AA0000400FA0500ED00E094110020704770B575
:106AB00005000DD002202C462034A073284601F09A
:106AC00017FA284600F0BEF80020A073607370BD6E
:106AD000012070BD7047704710B50446006801681A
:106AE000C943C90708D18168C943C90704D1012135
:106AF00041602046FFF76AFF20680168C9438907A3
:106B000008D48168C943890704D402214160204622
:106B1000FFF75AFF20680168C943490708D4816814
:106B2000C943490704D404214160204600F0DEF83F
:106B300020680168C943090708D48168C943090767
:106B400004D4082141602046FFF7B0FF20680168A7
:106B5000C943C90608D48168C943C90604D41021B1
:106B600041602046FFF731FF20680168C94389066C
:106B700008D48168C943890604D420214160204695
:106B8000FFF7A9FF20680168C943490608D4816856
:106B9000C943490604D4402141602046FFF79AFFCB
:106BA00010BD0000F8B5040005D025462035A87BAF
:106BB000002802D006E00120F8BD002068732046BE
:106BC00000F052F80220A8732068C2688446636807
:106BD000012B04D00120A16AC005814201D11E20F1
:106BE000824315486169814201D01448024014482B
:106BF000A668024018463043676A266A3E4330431F
:106C0000A66A30431043012B03D00122D2059642DD
:106C100003D12369E2681A431043074A914205D021
:106C2000A2691143E2690243084610436146C86005
:106C30000120A8730020F8BDFFFF00003F1FFFFFE9
:106C4000F8F119FF10B500680549884207D10548D9
:106C5000816B4900490881630D2000F055F810BD93
:106C6000007C00400010024010B5006808498842CE
:106C70000CD10848816BC2041143816300220121B9
:106C80000D2000F055F80D2000F048F810BD000070
:106C9000007C0040001002400068C069704700009E
:106CA00070B50224034620339C730F4C2568E6041C
:106CB000354325600468E568B6123543E56005682C
:106CC000AE6801242643AE6005682E6926432E6116
:106CD0000568A96101684A610068016904221143DD
:106CE00001619C73002070BD0004014070470000EA
:106CF0000448416B012211434163816B020411433B
:106D00008163704700100240C106C90E012088400F
:106D1000014908607047000080E100E0C106C90E2B
:106D200001208840014908607047000000E100E050
:106D300010B501F0A9FA10BD02494A6882434A60C1
:106D4000704700000070004002480168821511433E
:106D5000016070470070004002494A6802434A607F
:106D6000704700000070004005480168022211438E
:106D700001600448016904221143016130BF70477A
:106D80000070004000ED00E00A4B1A689208920083
:106D900002431A600848036904221343036101296E
:106DA00006D040BF20BF20BF0169914301617047F9
:106DB00030BFF9E70070004000ED00E0F8B5044690
:106DC0000078544D800672D5524E0027403EB06B7D
:106DD000C00004D4B06BA9050843B06301274E4836
:106DE0000168C90511D40168821511430160FFF7DC
:106DF000B1FD009005E0FFF7ADFD0099401A642851
:106E000037D845480068C005F5D532680321090523
:106E100060680A400140914208D08103890F03292C
:106E200004D13168890301D50120F8BD2A69032105
:106E300009040A4022D0084090421FD020788006E2
:106E40001CD528692A6988430121C9040A432A619B
:106E50002A698A432A612861C0050FD5FFF77AFDA8
:106E6000009008E0FFF776FD0099411A2B48814217
:106E700001D90320F8BD28698005F3D5616888032E
:106E8000800F032805D132680005824301400A4380
:106E900032602869032261681204114008432861A6
:106EA000002F04D0B16B012000078143B16320782B
:106EB000C00705D0E868A168800880000843E86042
:106EC0002078800705D5E8680C218843E1680843ED
:106ED000E8602078400706D5E868032189028843E6
:106EE00021690843E8602078000706D5E868032197
:106EF0000903884361690843E8602078000606D5E5
:106F0000E868032189048843A1690843E8600020F8
:106F1000F8BD0000401002400070004088130000DF
:106F2000F8B50E4605007DD053480068C007C00F75
:106F3000B0420AD250480168490849003143016013
:106F40000068C007C00FB04271D128784B4C800751
:106F500005D5E068F0218843A9680843E0602878F7
:106F6000C00752D06868022817D0032818D02168BB
:106F7000012818D08905002959DAE16889088900B3
:106F80000143E160FFF7E6FC69680746022912D079
:106F900003291CD0012926D033E021688903EAE7C0
:106FA00021688901E7E74907E5E7FFF7D3FCC11B43
:106FB0003348814223D8E0680007800F0228F4D1CB
:106FC00023E0FFF7C7FCC11B2D48814217D8E068BA
:106FD0000007800F0328F4D117E0FFF7BBFCC11BAB
:106FE000274881420BD8E0680007800F0128F4D1C0
:106FF0000BE0FFF7AFFCC11B2148814201D9032000
:10700000F8BDE0680007800FF3D11B480168C9078D
:10701000C90FB1420DD901684908490031430160E7
:10702000006800E003E0C007C00FB04201D00120BB
:10703000F8BD2878400706D5E06807210902884393
:10704000E9680843E0602878000707D5E068072171
:10705000C90288432969C9000843E06000F036F896
:10706000E168084A0906090F515CC84006490860F2
:107070000020FFF791FCF8BD002002400010024004
:1070800088130000B2A60008EC000020044805495F
:107090000068C968044A4905490F515CC8407047F7
:1070A000EC00002000100240CBA60008044805496F
:1070B0000068C968044A8904490F515CC840704798
:1070C000EC00002000100240CBA6000810B5184AC2
:1070D000D1680C20084004280BD0082810D00C28B8
:1070E00010D050680004410F0120C003491C8840A3
:1070F00010BD1068C00601D50E4810BD0E4810BD69
:107100000E4810BD88020E4B000F185C0902D368B0
:10711000890F491CDB0301D5084A05E01268D20635
:1071200001D5044A00E0044A5043FDF7E1FF10BDD9
:107130000010024000093D000024F40000127A0013
:10714000C2A60008FEB505007ED0FE4CE7680C2004
:10715000E66807400120000406402878C00747D0B1
:10716000082F05D00C2F0AD101200004864206D139
:10717000206880033CD568680028E5D038E001200D
:1071800069680004814203D121680143216011E054
:10719000052301221B0492049942216802D1114364
:1071A0002160F1E78143216021680140009120685E
:1071B00090432060686800280DD0FFF7CBFB00905B
:1071C00005E0FFF7C7FB0099401A64287AD82068C9
:1071D0008003F6D50CE0FFF7BDFB009005E0FFF75C
:1071E000B9FB0099401A6428F0D820688003F6D4CF
:1071F0002878800755D50923E868042F0DD00C2F77
:1072000001D1002E09D000283BD0216899430143C9
:107210002160FFF79FFB064627E02168490701D55B
:10722000002891D061681F22120291432A6912023C
:10723000114361602168994301432160FFF746FFD4
:10724000E16809060A0F00E079E1BF49895CC8409E
:10725000BE4908600020FFF79FFB002872D120E0A4
:10726000FFF778FB801B0228B0D820684007F7D5CD
:1072700060681F2109028843296909020843606088
:107280000FE02068400840002060FFF763FB0646DF
:1072900004E0FFF75FFB801B022897D820684007B7
:1072A000F7D42878C0065FD5002F0CD0A869002835
:1072B00049D02068FF21013108432060FFF74AFBD5
:1072C00006462DE0C0E02068800502D5A8690028A8
:1072D000A7D06068072149038843296A0843606092
:1072E0006068297F0002000A090608436060286A76
:1072F000410B0120C003491C8840E16809060A0FC0
:107300009149895CC840914908600020FFF744FB1F
:10731000002817D128E0FFF71DFB801B0228A3D807
:1073200020688005F7D56068072149038843296AEA
:10733000084360606068297F0002000A090608436C
:10734000606011E0E1E02168FF20013081432160AD
:10735000FFF700FB064604E0FFF7FCFA801B02285B
:1073600072D820688005F7D42878794E000724D594
:1073700068690028306910D0012108433061FFF7A7
:10738000E9FA009005E0FFF7E5FA0099401A0228B3
:107390005AD830698007F6D50FE0400840003061C8
:1073A000FFF7D8FA009005E0FFF7D4FA0099401AE9
:1073B000022849D830698007F6D42878400765D577
:1073C00000200290A06BC00006D4A06B0121090729
:1073D0000843A063012002905E480168C90511D4EA
:1073E0000168821511430160FFF7B4FA009005E0CF
:1073F000FFF7B0FA0099401A642825D8554800686C
:10740000C005F5D5FF20AA680130824203D1316959
:107410000143316111E001218902002A07D00523CF
:107420001B029A4203D132690A433261EFE73269A3
:1074300082433261306988433061A86800280FD0E8
:10744000FFF788FA009007E05EE0FFF783FA009903
:10745000411A4148814257D830698005F5D50DE081
:10746000FFF778FA009006E0FFF774FA0099411AE6
:107470003948814248D830698005F5D402980028FF
:1074800004D0A06B012109078843A063686A002823
:1074900064D00C2F3ED0012636060228206805D085
:1074A000B0432060FFF756FA05462FE0B043206056
:1074B000FFF750FA074604E0FFF74CFAC01B02281A
:1074C00022D820688001F7D4E96AA86AE2680843F4
:1074D000296BFD231B049A4311430843E060206895
:1074E00030432060FFF736FA054604E0FFF732FA32
:1074F000401B022808D820688001F7D52EE0FFF74E
:1075000029FA401B022801D90320FEBD2068800112
:10751000F5D423E00128F8D0E06801210904AA6A23
:10752000014091420BD10F218904EA6A0140914246
:1075300005D1032189050840296B88420ED001201E
:10754000FEBD000000100240B2A60008EC000020C2
:107550004010024000700040881300000020EFE758
:1075600070B5040007D0002625464035A662687C29
:10757000002802D005E0012070BD2E74204600F0E6
:107580002FF802206874206801684022914301604E
:10759000A168606822690843E16811430843616992
:1075A00001220843A169520211400843E1690843DE
:1075B000216A0843A16A084321680860A069042180
:1075C000000C0840616A0843216848602068C1696E
:1075D00092009143C161666501206874002070BD0E
:1075E00010B586B0044614216846FDF7E0FD104949
:1075F0002068884219D10F48416B821411434163BE
:10760000C16A01221143C162C06A00211040059085
:10761000E020009002200190032003900291049149
:10762000052069460007FFF7C9F806B010BD000045
:107630000030014000100240094910B5401E884248
:1076400001D9012010BD074C60610321081F00F023
:107650001BFE0020A06107202061002010BD00005B
:10766000FFFFFF0000E000E070477047F8B50268D8
:107670000446D0691168936805072D0F5BD0DD07BC
:10768000ED0FFF2621360E402E4367D0C60706D0E9
:10769000CE0504D501261662E26F3243E267870702
:1076A00002220426002F06DADF0704D027683A6298
:1076B000E76F3743E767470706D5DB0704D0236842
:1076C0001E62E36F1343E367020709D520220A40D5
:1076D0002A4305D0236808221A62E36F1343E36745
:1076E000E26F002A2FD0800606D5880604D5216EC9
:1076F000002901D020468847E06F21688968490643
:1077000001D4000724D5204601F09CFD2068816843
:10771000490619D58168402291438160E06E0028B6
:1077200012D020498163E06EFEF7AEFE00280AD039
:10773000E06E816B06E0850610D58D060ED5216EB4
:107740001CE020468847F8BD2046FFF78EFFF8BDB5
:107750002046FFF78AFF0020E067F8BDC50208D584
:107760005B0206D50120000510622046FFF77CFF72
:10777000F8BD030605D50B0603D5616E0029E0D1DF
:10778000F8BD4006FCD54806FAD5136820464021CE
:107790008B431360202161670021616600F069F965
:1077A000F8BD0000A191000810B5040003D0606F7F
:1077B000002802D007E0012010BD002170200155F3
:1077C000204600F027F824206067206801684908F7
:1077D00049000160204601F07FFD0128ECD0606A7D
:1077E000002802D0204601F0BDFB20684168092234
:1077F000D20291434160206881682A2291438160CE
:1078000020680168012211430160204601F010FC4C
:1078100010BD0000F0B587B0064614216846FDF79C
:10782000C6FC2C493068884251D12B48416B01225B
:10783000920311434163C16A01221143C162C06ACC
:1078400000251040059003204002009002200327ED
:1078500001A9A1C104200490052069460007FEF794
:10786000ADFF1F4C1D48A560E56081C48027E56021
:10787000A7602020256160610002A0611848083CD3
:10788000FEF77CFE002801D0FEF778F9F466A662C8
:10789000144C1248214614382060032060601020E8
:1078A0000831A1C16561A561E56120462562FEF749
:1078B00065FE002801D0FEF761F9B46600220121BF
:1078C0001B20A662FFF734FA1B20FFF727FA07B048
:1078D000F0BD0000003801400010024030000240BE
:1078E00090150020D8150020F8B50446806F202898
:1078F0004DD100290BD0002A09D00123A0681B0319
:10790000984206D12069002803D1C80701D0012080
:10791000F8BD25466035287C012838D00120287420
:107920005820616502530026E6672220A067E06EBA
:10793000002819D01749C162E16E17480863E16E4B
:1079400016484863E06E13468663676D21683A46C1
:107950002431E06EFEF75AFE002805D01020E067C3
:107960002E7420206067D2E72E7420680168FF2201
:107970000132114301602068816801221143816056
:10798000206881684022114381600020F8BD0220F8
:10799000F8BD0000FD9100083B920008B591000879
:1079A00070477047FFB50446406F83B017460D46D9
:1079B00020285CD1002D0AD0002F08D0A168C0017A
:1079C000814207D12069002804D1E80702D00120B4
:1079D00007B0F0BD204660300290007C012846D000
:1079E0000298012101740020E06721206067FEF702
:1079F000B1FF264640360190378277820120A16888
:107A00000003814202D12069002802D02F460025C0
:107A100011E000270FE000228021204601F070FDD8
:107A2000002815D1002F15D02168387888627F1C76
:107A3000708A401E7082708A019B00280698009010
:107A4000E9D100224021204601F05AFD002808D04B
:107A50000320BDE728882168C005C00D8862AD1CE1
:107A6000E6E720206067029900200874B0E7022052
:107A7000AEE7704701490248C160FDE70400FA051E
:107A800000ED00E010B50524240700220421204663
:107A9000FEF759FF002208212046FEF754FF0A2076
:107AA00002F02BF8012204212046FEF74CFF0A20A9
:107AB00002F023F8002204212046FEF744FF10BD07
:107AC00010B505242407002204212046FEF73BFFC1
:107AD000012208212046FEF736FF0A2002F00DF8A9
:107AE000012204212046FEF72EFF0A2002F005F8AD
:107AF000002204212046FEF726FF10BDF8B5002421
:107B00000526074625463607002204213046FEF7A3
:107B10001AFF0A2001F0F1FF012204213046FEF78E
:107B200012FF6006040E08213046FEF703FF00280E
:107B300001D0641CE4B2052001F0DFFF6D1CEDB242
:107B4000082DE1D3002F03D0FFF79CFF2046F8BD9E
:107B5000FFF7B6FFFAE770B505260546360700229F
:107B600004213046FEF7EFFE0024E80901D001228F
:107B700000E0002208213046FEF7E5FE6806050E0B
:107B80000A2001F0BAFF012204213046FEF7DBFE95
:107B90000A2001F0B2FF002204213046FEF7D3FE96
:107BA0000A2001F0AAFF641CE4B2082CDDD370BDEA
:107BB00010B505242407012208212046FEF7C3FE44
:107BC000012204212046FEF7BEFE002208212046A5
:107BD000FEF7B9FE0A2001F090FF002204212046A2
:107BE000FEF7B1FE10BD10B50524240700220421C4
:107BF0002046FEF7A8FE002208212046FEF7A3FE3D
:107C00000A2001F07AFF012204212046FEF79BFEA4
:107C1000012208212046FEF796FE0A2001F06DFFA2
:107C200010BD70B505252D07002401220821284626
:107C3000FEF789FE062001F060FF0122042128469C
:107C4000FEF781FE062001F058FF07E0641CE4B255
:107C5000FA2C03D9FFF7C7FF012070BD0821284681
:107C6000FEF768FE0028F1D1002204212846FEF725
:107C70006AFE002070BD0000F8B501F009FA01F0BD
:107C800043FA4C480068C0694B4E4C4F800700D502
:107C9000FE60FEF763F84A4C0246608849490028B6
:107CA00003D0401E608001200870087801218902FD
:107CB000454D00281CD0012804D0022804D00328F8
:107CC00006D115E0212A13D200222846FEF73BFEFA
:107CD0000121C9023C48FEF72DFE3C490025002841
:107CE00028D03B48056008468079002802D006E08D
:107CF0000122EAE735490120887101F045FC33484B
:107D00000078632806D9002208212F48FEF71BFEC1
:107D1000012205E0012208212B48FEF714FE002273
:107D200001210520C9030007FEF70DFEA08C0128E4
:107D300003D01CE08D710022EDE7264869460880DB
:107D400072B680212448FDF731FF002804D00222BA
:107D500069462148FDF7CEFF62B620A001F0B0FCD5
:107D6000A58402F027FC642001F0C0FEFE60608C58
:107D7000012809D1124865844038058002F01AFCB8
:107D8000642001F0B3FEFE60208C012806D125841A
:107D900002F010FC642001F0A9FEFE600848134ABE
:107DA00040380188914202D1C088002800D1FE608D
:107DB000F8BD0000101500200400FA0500ED00E0F9
:107DC000600D00205A00002000040050BC0000207C
:107DD000E4000020AAAA0000384A0008BDF8C8EB59
:107DE000C9FDBCB6C4A3CABD0D0A0000AA55000057
:107DF00008B53721202000F06EF80321212000F083
:107E00006AF84021222000F066F80821232000F0C3
:107E100062F8AA21302000F05EF80A4802210187AA
:107E2000322000F058F80121332000F054F85F218F
:107E3000202000F050F8684600F006F80A2001F013
:107E40005CFE08BD200D002010B501460F2000F09B
:107E500021F8002800D0012010BD10B50446FFF71E
:107E6000A7FE3220FFF777FEFFF7DBFEE0B2FFF759
:107E700072FEFFF7D6FEFFF79BFE3320FFF76BFE87
:107E8000FFF7CFFE0020FFF739FE0446FFF7ABFEF9
:107E9000204610BD10B50C46FFF7DFFF2070012013
:107EA00010BD70B50D460446FFF782FE3220FFF785
:107EB00052FEFFF7B6FEE0B2FFF74DFEFFF7B1FE50
:107EC0002846FFF748FEFFF7ACFEFFF78CFE0A20BE
:107ED00001F013FE70BD10B5FFF7E3FF012010BDE8
:107EE00010B50248FEF7F8FD10BD00008814002010
:107EF000FEB50446002572B60068394A831804D1DD
:107F00003849CD68032189040D4081680191C16819
:107F1000009141698669002B08D132484038836A54
:107F2000C7043B438362836ABB4383620846304392
:107F300048D02B482368C34205D12A48C36803228E
:107F400092049343C360002917D02068026901237B
:107F50001A43026120684161FEF7FCFC0746FEF708
:107F6000F9FC2168C01B0968090703D47D21C900F9
:107F70008842F4D9216808204860002E17D0206874
:107F8000016901221143016120688661FEF7E2FC6C
:107F90007D270646FF00FEF7DDFC2168801B09688F
:107FA000C90601D4B842F6D92168102048600C48AF
:107FB0002168C14206D10B48C16803229204914353
:107FC0002943C160206801694908490001612168AD
:107FD0000198886021680098C86062B6FEBD000004
:107FE0000084FFBF401002401CB5002116480091DC
:107FF000144A01910260C163120542608160072248
:108000008263012202610246C16020321170FF23A7
:108010005170C23343628162117301638161042232
:1080200041634261C161FEF795F8084800908013F2
:10803000019069460448FEF73DF800210248FDF72B
:10804000E3FF1CBD002401402C14002002000004AA
:1080500008B50848016B012211430163006B01213F
:108060001040009000220A20FEF762FE0A20FEF770
:1080700055FE08BD00100240F0B587B014216846D7
:10808000FDF795F84C48C26A04210A43C262C26AED
:108090000A400592C16A80273943C162C16A3940EA
:1080A0000591C16A01252943C162C16A2940059130
:1080B000C16A02263143C162C06A2A463040059037
:1080C00005201C210007FEF73EFC01223B493C48ED
:1080D000FEF739FC00223B493948FEF734FC912178
:1080E0000520002209020007FEF72DFC364801900A
:1080F000002405206946009502940007FEF75EFB08
:108100000320019005206946009602940007FEF7BF
:1081100055FB0C20009011200190032003900520B6
:10812000029469460007FEF749FB102000900520E5
:1081300069460396019502940007FEF73FFB112064
:10814000019002946946009503941D48FEF736FBA2
:108150001E4801906946009602951948FEF72EFBCD
:108160001B48009002946946019503941448FEF759
:1081700025FBE8026A4651C269461148FEF71EFB1C
:108180009120000200900520029469460195039415
:108190000007FEF713FB6946094800970295019412
:1081A000FEF70CFB002201210520FEF7C1FD052092
:1081B000FEF7B4FD07B0F0BD00100240010600005C
:1081C00000040050083000000000111000002110D1
:1081D0000836000010B50F4C0D482060FF20053018
:1081E00060600020A060E06020616061E0610121CA
:1081F000206249026062A161A0620720E06220461D
:10820000FFF7AEF92068016840221143016010BDFC
:1082100000300140B814002000B585B01421684634
:10822000FCF7C5FF164815490160E121490241608C
:1082300000218160C160016181610C22C1614261E4
:108240000162302141620121090381634900C16358
:10825000FFF7AAFA0120800200900220019001207D
:108260000290032003900420049005206946000733
:10827000FEF7A4FA01F082F905B000BD0038014014
:1082800010150020704700008307FF22DB0E9A4084
:108290008907090E994000280BDA0007000F0838FB
:1082A000830808489B001818C36993430B43C361B4
:1082B0007047830804489B001B18186890430843C4
:1082C0001860704700ED00E000E400E0BFF34F8F5E
:1082D00004490348C860BFF34F8F00BFFDE70000AB
:1082E0000400FA0500ED00E0F0B585B00A2001F0C9
:1082F000E1FE002001F0F8FEF84D0024AC70A87BF0
:108300000C2801D30B20A87301220520510200077D
:10831000FEF719FBEC70F248AC74F24E0078307145
:108320000221F148FEF706FB002860D00020A97961
:10833000EC4E49000843F071A86AF070401CA86236
:1083400068793146B0724200B4310846A938FCF76A
:1083500015FF0620707230461338297F0175697F3A
:10836000417568790022400031460D3001F08CFFE4
:108370006879002140000D3001F098FF022001F0E3
:10838000E9FE0024F4712C74AC7201202873EC72A5
:10839000D648FEF781FC28840646EC706879FDF724
:1083A0006DF9D34AD34BFDF763F801F03BFB012392
:1083B00000229B07FCF7AAFFFDF7A6F90006C10CF7
:1083C000881980B20121C9036884884201D3401A08
:1083D0006884C94868632879401C2871C348FEF73F
:1083E0005BFCE883BF48C54C4E30029071E1012030
:1083F0009DE7BE48FEF750FCE883C14F0AE0BB484A
:10840000FEF74AFC80B2E883698C884202D30919DE
:10841000884206D300210F2001F0CCFD3842E862EB
:10842000EDD0E86A411C20D02E4640047ED5812242
:10843000D20100210F2001F0FCFE002001F054FECB
:10844000002001F006FE0021102001F0B3FD4106DE
:10845000A448490E00225030019101F0E1FDA148ED
:108460005030417A0729C1D101E0FFF72FFF9D4825
:108470000222A4495530FCF7A5FE0028B6D101F030
:1084800066FFF164B06401F04FFF71653065F0780C
:108490009449401CF0704D310A7968460270497960
:1084A00041700088B18B88427ED10298964F008A35
:1084B00038808C484C30808A30838C48FEF7ECFB47
:1084C000F083308B9149FF30C33080B230838842D3
:1084D0000CD949424018308338888C49401C80B2FE
:1084E0000B313880884201D30020388002987B4AC3
:1084F00081891186C0895086326B7263794A503205
:10850000D27C13071B0F032B00D0B3741209F27433
:10851000002333710123B372704B002A9986D886E9
:1085200015D0704802227749553000E0C5E0FCF7CD
:1085300049FE00280BD101206A493074C8710198A6
:1085400064311638C2B272747148FCF717FE01200C
:10855000F07264496148042251314030FCF70EFE4C
:108560006048736D1630326D01F0C6FE3F887D2085
:10857000C000318B78434018B0630490654801789F
:10858000F17365480191C088FDF75DF800903846A9
:10859000FDF759F80099FCF77BFE7F21C905FCF730
:1085A0001EFEFDF779F800E02BE05A4980B2088002
:1085B0000199491E884201D10120F072B78414202C
:1085C000305EFDF747F801910090F08BFDF756F80B
:1085D000524A534BFCF74CFF074603910498FDF7B2
:1085E00039F83A46039BFCF735FF019B009AFCF7EC
:1085F0008DFEFDF765F8F0634A48008800F0B6FB91
:1086000067E0FDF793FB0746414803210C38C1554D
:108610000298324982890A86C08948863C4AB80055
:108620009C3A316B11502F49736D40181A30326DDE
:1086300001F062FE70797F1C87424AD101F0D8FBBD
:10864000FF23296D5B04686D0022C91850410006A4
:108650000C0A044360084000010E0002E965A865A9
:108660002048EB6C0A30AA6C01F046FE1D48EB6D09
:108670001230AA6D01F040FE1A4808214172687953
:108680000022800017491C3001F0FEFD68790021AE
:1086900080001C3001F00AFE204601F004FD01209C
:1086A00001F058FD0006000E287240D100210F2075
:1086B00001F080FC0006F9D539E03A4600210F2090
:1086C00001F0B7FDF0787179884202D0002001F006
:1086D000C0FCE98B688C814226D28AE648000020E3
:1086E000BC000020941100200004005088140020D9
:1086F000B81E85EB51B8CE3FA0860100983A000025
:1087000000D02724D8000020E0000020E70300006C
:1087100014130020D4000020200D0020F853E3A5FE
:108720009B843E40C400002000198142D5D86D4A88
:1087300000210F2001F07DFD6B4800240078002807
:1087400003D16A48008800F011FB002768493846C9
:108750008F734A79039221E0634B195C00291BD087
:10876000634DA300AE7B9C46761CAE735E4D6600E7
:10877000303DE9505C4B4500C03B5D5B18339D5379
:1087800085001833584E5D596346603EF550641CB1
:10879000554B491EE4B21954401CC0B29042DBD381
:1087A0005348C178032901D2817B8173504900224B
:1087B000887B4873401E35E000212FE04A4D8B0036
:1087C000603DEC585E1901967668B446644523DD39
:1087D00000944C00483D2D5B9600AE46424D303D26
:1087E000AD59414E02956546603EF5503546483DCF
:1087F0006519AC466D88483E3553344678341E19A9
:10880000394D7468303DEC50019C009B63607546A7
:1088100063465D80029D7560491CC9B28142CDDB13
:10882000521CD2B28242C7DB2F48603802683048FF
:10883000416B32398A421ADA2B49303909680029EA
:1088400015D0C179491CCAB2C271032A05D9264A7A
:10885000A83A12888283012202700179032900D983
:108860000770214B00210478C03B039A08E0C771D0
:10887000F3E74D005D5B002D00D10124491CC9B216
:108880009142F6D3184B00211A4A0470903B8C0099
:10889000491CC9B21A510C29F9D3007C002806D012
:1088A00011490C3108784B788A7802280ED00D4A8D
:1088B000002180320F2001F0BCFC012105200022A4
:1088C00049020007FEF73FF805B0F0BD0A48C91C91
:1088D000C018FCF753FC01F06DFE642001F006F9AE
:1088E000C3E5000000D0272408130020C4000020A6
:1088F00048000020FFFF0100200D0020704700000D
:10890000F0B589B0934800900020C0430590002640
:108910000A2001F0CFFB002001F0E6FB00208E4C86
:108920000546A0708D4F8E4806908D480022C238B3
:1089300085730146142001F0A7FC0021142001F0EA
:10894000B5FC022001F006FC00210F2001F032FBF3
:108950003842E062F8D0E06A411C18D040047DD56E
:108960008122D20100210F2001F063FC00211020A0
:1089700001F020FB41067A48490E0022801C01F0DC
:108980004FFB7748801C417A022902D0C1E0FFF7F3
:108990009DFC734802227349C01DFCF713FC00289C
:1089A000F4D101F0D4FCE164A06401F0BDFC616588
:1089B0002065002E22D106996B48098A01806848FB
:1089C0000126801E808A20836848FEF765F9E083CF
:1089D000208B6749FF30C33080B2208388420DD995
:1089E00049424018604920830888614A401C80B28F
:1089F0000B320880904201D3002008800698694617
:108A000082898A80C089C88055490422C91C0846C9
:108A1000A238FCF7B3FBFF22216D5204606D0023E6
:108A2000891858410006090A01430846029101F0DD
:108A30003AFB029948084000010E0002E165A0657A
:108A40004748E36C9638A26C01F056FC4448636DCD
:108A50009238226D01F050FC414800E05BE08E3816
:108A6000E36DA26D01F048FC3D490022A0393C2095
:108A700001F00AFC00213C2001F018FC012001F06B
:108A800069FB2072A0780121401CA0700520C90359
:108A90000007FDF75FF9206CFDF70AFA02903548F0
:108AA00001880298FCF724FB33480088414388B2D0
:108AB000324908800299491E618300F057F90199F3
:108AC000009881420DDA00290BD025490422C91CE7
:108AD00005A8FCF753FB0120207005206072019867
:108AE0000090207A002805D100210F2001F062FAC1
:108AF0000006F9D5802200210F2001F09AFB00200A
:108B00006D1CEDB26070032D00D20EE7002E08D070
:108B10001BE00120F4E71A4A00210F2001F089FB35
:108B2000F7E7608B401E0004000C608303D01149FE
:108B30000988884202D90F48018861830E49608BF9
:108B40000988401E48430D4908800598A08309B054
:108B5000F0BD00003F420F004800002000D0272455
:108B6000E2110020D8000020E0000020881400203E
:108B7000E7030000C8000020C6000020C400002059
:108B800000902724F8B52D492B48086001F0B2FC6D
:108B90002C4D2B486880E888002801D16420E880AB
:108BA00029480178432901D943210170E98E0170D8
:108BB000264CE88F2071A88F6071A87AA070AE88CB
:108BC0000521E6616181EF883846FCF791FAA081C2
:108BD00001463046FCF78CFA8800081886B27D20E2
:108BE000C00026817043FCF749FD194A194BFCF778
:108BF000A7FCFCF789FDE0817D2066823946C00034
:108C0000FCF776FA2082E08201202083FDF7A6F8A7
:108C1000A082E28910491148FEF742F810A0E169EC
:108C200000F04EFDE98812A000F04AFD298915A048
:108C300000F046FDF8BD0000B59500084400002096
:108C400003020000200D002000000020BC000020D6
:108C5000F853E3A59B843E40FF7F0000881400206A
:108C6000B1EAC7A949443A202564202E0D0A000024
:108C7000CDA8D1B6BCE4B8F43A202564206D732E9B
:108C80000D0A0000B5A5B4CECDA8D1B6BBF9D5BEAE
:108C9000CAFDC1BF3A202564B8F62E0D0A000000B7
:108CA00070B586B014216846FCF781FA01250F4E95
:108CB000ED03002229463046FDF745FE0120002441
:108CC000019002946946009503943046FDF776FDC5
:108CD0000320019002946946009503943046FDF705
:108CE0006DFD022000F002FF06B070BD00040050D0
:108CF00070470000F8B5044600206A461080194D00
:108D000055222A70AA226A700322AA70661DEE708C
:108D10002A716971144A49008918AC712246E81D0C
:108D2000FCF72CFA002007E029186A468978128897
:108D300089186A461180401CB042F5DB611DA81CF1
:108D4000FCF778FE01466846018029190078C87151
:108D500068464078087221460931024800F08AFAD4
:108D6000F8BD0000C8130020200D002010B51349E5
:108D70000A8BCB8A9A4201D3D21A0A83104A098BF2
:108D8000D2884A437D211018C90048430D4909681B
:108D9000401AFCF75FFC0C4A0C4BFCF7D1FBFCF7CC
:108DA0008FFC0B49884201DD4A428018002800DA16
:108DB000401808490968486110BD0000BC00002047
:108DC000200D002084000020F853E3A59B843E4042
:108DD000FF7F000088140020034A1168382389B2FD
:108DE00099430143116070470030014010B5FDF711
:108DF000B7FD10BD10B59AB034216846FCF7D7F91D
:108E000014210DA8FCF7D3F91C2112A8FCF7CFF907
:108E10001B4801680324E402A143C21489180160BD
:108E2000FDF792FF17480169A143016106200090F8
:108E3000FF200130029001200390102004900220B6
:108E4000099040040B90000100240C900A9468469D
:108E5000FEF778F90F200D9003200E900F941094D8
:108E6000012111940DA8FEF75BF8812012900320D8
:108E700080041890149412A8FDF7A0FF1AB010BD3A
:108E800000700040401002401048016882151143F4
:108E90000160C1680E4A1140C16001680D4A11406D
:108EA00001608168490849008160016801229204DB
:108EB00091430160C168FD2212049143C160002109
:108EC00001610649044888607047000000100240B4
:108ED0000C40FF88F6FFF6FE0050000800ED00E0B1
:108EE00070B501F07BF81D4C1D4D606402E001F08F
:108EF00075F86064A842FAD1207801250526ED03B3
:108F00003607002804D001280FD0022823D120E002
:108F1000012229463046FDF716FDFFF7F1FC00223D
:108F200029463046FDF70FFD15E0607A0122401E0C
:108F3000607229463046FDF706FDFCF72BFF002244
:108F400029463046FDF7FFFC607A002803D12070E7
:108F500001E0FFF7C9F900F033FF70BD48000020C1
:108F60003001CADE10B5818CC90707D001684A6894
:108F700001235B049A43836A1A434A60818C890700
:108F800007D501684A6801231B049A43C36A1A4340
:108F90004A60818C490707D501684A6801239B0410
:108FA0009A43036B1A434A60818C090707D501680D
:108FB0004A680123DB039A43436B1A434A60818C5E
:108FC000C90607D50268916801231B039943836B87
:108FD00019439160818C890607D501688A6801234D
:108FE0005B039A43C36B1A438A60818C490612D58E
:108FF00003685A6801210905046C8A4322435A60B8
:10900000026C8A4207D10268516803235B059943C9
:10901000436C19435160818C090607D501684A6881
:109020000123DB04806C9A4302434A6010BD0000B8
:10903000F8B500260446C667FDF78CFC0546206897
:109040000068124F000709D501212B46002249056F
:109050002046009700F054FA00280DD120680068DF
:1090600040070BD501212B46002289052046009799
:1090700000F046FA002801D00320F8BD20206067E8
:10908000A067603426740020F8BD0000FFFFFF01D8
:10909000F8B5184CC826E078002829D16079002856
:1090A00026D101206071144D686B002700281ED066
:1090B000686BC821081A15E01048E168405C6169D6
:1090C00088470F480A21008848430E490880E06815
:1090D000401CE060E068C82800DBE760696BC820DE
:1090E000401A761EE168814201D0002EE4DC6771EF
:1090F000F8BD00003000002000000240580C0020A5
:10910000CC000020D600002070B5224CE07800286A
:109110003FD1207900283CD1012020711E4EF169F9
:1091200000250906002933DA2156625791420AD1F7
:10913000F06940062CD5A079002829D0A571208996
:10914000401C208124E0A179002903D1A0710A20CC
:1091500000F0D3FC00202056CC2148430F49421890
:10916000206912181279B262401C00222061A256B6
:10917000CC235A43895881420ADC25612078401C5F
:10918000207020780E2800D12570A078401CA07097
:10919000257170BD300000200038014030010020F2
:1091A00010B5806A0022014640314A834A82FEF7A8
:1091B0005CFA10BD70B5846A606FA56F216889681C
:1091C00000260906002906DA212804D15220065378
:1091D000204600F047F820688068400606D5222D1A
:1091E00004D15A200653204600F02CF8E06F1021DD
:1091F0000843E0672046FEF738FA70BD10B5014617
:109200000968806A0968890614D400225A210A5222
:1092100001680A68FF2301339A430A6001688A687B
:10922000520852008A6001688A6840239A438A6023
:1092300020218167FEF7B4FB10BD10B5806AFEF7F0
:10924000B0FB10BD01680A68FF2321339A430A600E
:1092500001688A68520852008A60202181670021D3
:109260000166704701680A68C0239A430A6020219A
:109270004167704770B5164CE278002A0CD122790C
:10928000002A09D10122E2700025C82903DC02224C
:10929000A256002A01DCE57070BD0123E356CC2202
:1092A00053430C4AD1500123E356CC2673439B18F9
:1092B0000A460146181DFBF761FF6078401C60708C
:1092C00060780E2800D16570A078401EA070E2E79B
:1092D0003000002030010020F8B504462669A2685D
:1092E000E76932436669102000253E432368324314
:1092F00078491E68784F3E4016431E6023685A68BE
:1093000003263603B243E66832435A602368A269F3
:109310008B4201D0266A32439E680B273F02BE4330
:1093200016439E606D4E23686D4AB3420CD1D268DD
:109330009207920F06D0012A38D0022A34D0032A8D
:1093400020D11EE001201DE0664EB3420AD1D26852
:109350000C26324026D0042A28D0082A24D00C2AF1
:1093600010D10EE08B420DD1D66803229202164036
:1093700018D001229202B61A18D0B61A14D096420A
:1093800000D10820564A0126403A574FF6038B4237
:1093900036D100280CD002280DD0042812D008287D
:1093A0001FD11CE00020EDE70220EBE70420E9E7F5
:1093B000FDF76CFE08E01068C00601D5384605E0F0
:1093C0004A4803E0FDF782FE002873D0626851002E
:1093D0005118814205D81103814202D303E030467F
:1093E000F4E7012566E0010E06025008002330185C
:1093F0005941FBF793FE03210902411A3C4A55E00B
:10940000E169B14232D1030000F081F909070A0D88
:1094100006250606062B0600E3E7FDF737FE1CE0EF
:10942000FDF744FE19E010686168C00602D54808DF
:10943000304A01E0304A48088018FBF759FE80B2F4
:1094400001462E4A10399142CBD8511C01400007E9
:10945000400F08432CE0FDF739FE616840004A08E0
:10946000EAE76168012248081204E5E7030000F01A
:109470004EF909070A0D06260606062C0600B0E777
:10948000FDF704FE1DE0FDF711FE1AE010686168AB
:10949000C00602D54808C01902E014484A0810184E
:1094A000FBF726FE80B20146144A1039914298D843
:1094B0002168C8600020206660662846F8BDFDF778
:1094C00005FE61684A088018EAE761684808801963
:1094D000E6E7000000480040F369FFEF0038014074
:1094E000401002400044004000093D000024F40008
:1094F000FFFC0F0000127A000048E801EFFF0000B7
:10950000FFB581B017460E4604460A9D09E0681C67
:1095100007D0FDF71FFA0499401AA8420CD8002D75
:109520000AD02068C1693046884318D00020B8426C
:10953000EDD0002005B0F0BD20680168FF22A13207
:1095400091430160206881684908490081602020BA
:109550006067A0670020603420740320EAE70120E0
:10956000E5E7000010B504491020096808620248C8
:10957000FEF77CF810BD00001015002001490D20F9
:10958000887070473000002010B507480A22018A11
:1095900051434183FEF75CFDFEF73EFEC8220349BE
:1095A0000348FEF7A1F910BDBC000020580C0020B4
:1095B00010150020F8B53D4C002321783C4A1D468B
:1095C000082910D0072945D006294ED0052950D0AA
:1095D000042951D0032952D0002954D0012956D052
:1095E000022958D059E0A17800264A1F04E0304FE4
:1095F000BF5DFB189BB2761C9642F8DB6679277933
:109600009A195118E3786278C9188918C91940184D
:10961000C0071AD0012E14D0022E16D12548244995
:10962000C018FBF7ABFD00F0C5FF642000F05EFA48
:10963000BFF34F8F21492048C860BFF34F8F00BF51
:10964000FDE759081046FFF755FB2570E570A5703A
:10965000A571F8BDA1795054491CC8B2A071A17878
:10966000491F8842F5D1082001E060700720207072
:10967000F8BDE0700620FAE760710520F7E7A070FA
:10968000E5700420F3E7552807D10120EFE7AA2869
:1096900003D10220EBE7032803D02570E570A57005
:1096A000F8BD032020702071F8BD0000B300002039
:1096B00064130020200D00200400FA0500ED00E0F6
:1096C0000FB410B503A9044B044A029800F002F944
:1096D00010BC08BC04B0184711A30008F00000201B
:1096E0002021020C01D010211046020A01D01046A0
:1096F0000839020901D01046091F820801D010461E
:10970000891E420801D0881E7047081A704730B47D
:109710007446641E2578641CAB4200D21D46635D0E
:109720005B00E31830BC184702E008C8121F08C1EC
:10973000002AFAD170477047002001E001C1121FD2
:10974000002AFBD1704708B50021684601706B46BE
:10975000012202212C2000F07BFD022168460170CD
:109760006B4601222C2000F073FD08BD38B504467D
:109770006D20694608706B46012207492E2000F0D3
:1097800067FD0649002C01D0054A00E0054A2E205D
:1097900000F044FD38BD0000060800000618000077
:1097A000070600000716000038B504466B46022283
:1097B0000021362000F018FCB3212300FFF7A7FF9B
:1097C0000E0F08153A3A3A3A1C273A3A2F34483ADB
:1097D00000216846017040784108490014E069465C
:1097E000087880088000401C04E0694608788008FA
:1097F0008000801C08701DE0684602780A404832EC
:1098000002704178802001436846417012E068464A
:1098100002780A40027040784106490EF4E7694632
:1098200048780221084303E069464878FD21084052
:10983000694648706B4601220021362000F008FD81
:10984000012200AB11463620013300F001FD38BD86
:1098500069460878CF21084069462030CAE708B534
:10986000032168464170012101706B4602220021EC
:10987000362000F0EDFC0122D20306212D2000F05D
:10988000CDFC012000F032F90120FFF78DFF08BD6B
:1098900008B5020A69464A7008706B460222042124
:1098A0002D2000F0D5FC0320694608706B4601228C
:1098B00006212D2000F0CCFC0020694608706B4684
:1098C000012206212D2000F0C3FC0A212D2000F0EA
:1098D00071FB08BDFFB58DB00446002506E02528C4
:1098E0000AD0109A0F999047641C6D1C20780028AC
:1098F000F5D1284611B0F0BD00270121484A009754
:1099000000E00743641C23780846203B984010423F
:10991000F7D120782E2817D1042007436078641CE3
:109920002A280CD10E98641C02C800910E900BE0FE
:1099300000990A22514330394018641C0090207865
:10994000014630390929F3D920780028D1D064287C
:1099500008D0692806D075281ED0109A0F99904714
:109960006D1C5BE00A200E99019001C90E91002840
:1099700002DA40422D2102E0390504D52B216A4646
:109980001172012103E0F90704D02021F7E70BAEA3
:109990000B910DE00021FAE70A200E99019001C910
:1099A0000E91F7E70199FBF7A3FB3031761E31707A
:1099B0000028F7D103A8801B20300190780701D53B
:1099C000009801E0012000900199884201DD401AD1
:1099D00000E000200027009006E002A8109AC05D79
:1099E0000F9990476D1C7F1C0B988742F5DB04E0B4
:1099F000109A30200F9990476D1C0099481E0090D6
:109A00000029F5DC05E03078109A761C0F99904714
:109A10006D1C0199481E01900029F4DC641C65E767
:109A200009280100F8B54A002B4B520DD6182B4AD5
:109A30000C460546142E2BDA002E12DA284BFBF7C3
:109A400065FC00221346FBF78BFF40D2002C03DAA3
:109A50000124E40700253AE02046284337D0214C72
:109A600014E0214F0B46F7403B402B4331D01C4BB9
:109A7000FBF74CFC00221346FBF772FF27D2002CA9
:109A800003DD01200005F0400419BC4300251EE061
:109A9000332E1EDC33460027143BFF43DF403842A1
:109AA00017D00F4BFBF7DCFC00221346FBF758FFE7
:109AB0000DD2002C0ADD142E0CD03420811B012085
:109AC00088404019A84200D2641C0546BD43214687
:109AD0002846F8BD641CF9E701FCFFFF9C7500886F
:109AE0003CE4377E0000F03FFFFF0F007D2110B502
:109AF000C900484300F001F810BD002140E000BF5C
:109B000000BF00BF00BF00BF00BF00BF00BF00BF5D
:109B100000BF00BF00BF00BF00BF00BF00BF00BF4D
:109B200000BF00BF00BF00BF00BF00BF00BF00BF3D
:109B300000BF00BF00BF00BF00BF00BF00BF00BF2D
:109B400000BF00BF00BF00BF00BF00BF00BF00BF1D
:109B500000BF00BF00BF00BF00BF00BF00BF00BF0D
:109B600000BF00BF00BF00BF00BF00BF00BF00BFFD
:109B700000BF00BF00BF00BF00BF00BF00BF491C47
:109B80008142BCD370470000FEB50446002001901E
:109B900000906079734940000E5A61782578491E1B
:109BA0007148CFB20163042D77D0072D75D0002105
:109BB0000291217801736C49E37901229205896948
:109BC000002B6CD0914381616748217A4173217ADF
:109BD00082698907890B0A4382610021042000F011
:109BE00028FB324661492E2000F018FB3846FFF76B
:109BF000BDFD5F4E0522705D810040185D49431830
:109C000007212B2000F024FB5B49029801220B184E
:109C10000B21282000F01CFB705D584980000A5879
:109C20000C21282000F005FBE07955498000401800
:109C3000A1794900425A0221272000F0EFFA514849
:109C40007E00825B0421272000F0E8FAE0790028FA
:109C500029D0A07804282CD0282069460872202218
:109C60000621272000F0DAFA02AB01222621272064
:109C700000F0EEFA444938014018E1788900425872
:109C80000821272000F0D5FAA17A601C627A090227
:109C9000114313D016E000E001E0012188E71143F1
:109CA000F608816190E764220621272000F0B6FAC9
:109CB000E0E71020694608720246D1E73349017295
:109CC000090A4172417A007A0A02024320212720C0
:109CD00000F0A4FA2E4F0C2123203A6800F0A9FAD4
:109CE000F01982880421232000F098FAA079002836
:109CF0000BD0E0792749012243180021212000F0F0
:109D0000A7FA03200190012000902A07120F1001EA
:109D10000243607800218007000B02430198000590
:109D200002430098400402432079C00640090243E0
:109D30006079C00602431F2000F07BFAA0786178AA
:109D40000123084302040848DB030261E179490367
:109D500019430A4302610021082000F06AFA00203A
:109D6000FEBD000080A60008F400002004280000CA
:109D700028A60008010000201F00002030A60008CF
:109D800050A600085CA6000860A60008411000006C
:109D900048A600082100002038B50C4607498A8BE8
:109DA000002102432C2000F039FA684604706B460B
:109DB000012206212C2000F04BFA38BDF4000020CF
:109DC00010B5FFF7C0FC10BD10B5044604213620C5
:109DD00000F0F0F80121C902002C01D0084300E096
:109DE000884302460421362000F023FA10BD00000B
:109DF00038B540206946087000210E2000F0DAF8DE
:109E00000446002211460E2000F013FA6B46012290
:109E100000210D2000F01CFA074A00210F2000F05D
:109E200008FA00F0E1F9224600210E2000F001FAC4
:109E300002480021017338BDF8FF272414010020D7
:109E40007CB505460420694608704B4C00206075BF
:109E500021462031206348710873A0836063A063AA
:109E600000F0BCF8454E206002E000F0B7F820603A
:109E7000B042FAD10020FFF797FC4148007824282F
:109E800001D9243806E00621FBF732F90622101A20
:109E900040010843020601040A4301020A43024347
:109EA00000211E2000F0C5F96B460122002124206C
:109EB00000F0CEF91E20FFF7EBFC86B2300AA0734B
:109EC0000420FFF7E5FC0006000E0DD002206946D5
:109ED000087101AB012212212D2000F0B9F9A08BED
:109EE000012109030843A08300F078F820600620D0
:109EF000FFF7CEFC60600720FFF7CAFCA060F00609
:109F0000C00E207501D110202075C0B200F0DCF920
:109F1000E80707D0FFF7A3FCA08B0121C902084383
:109F2000A0830AE00521362000F02EF815490840EC
:109F300002460521362000F071F90120FFF734FCBC
:109F40000021042000F036F8A0610021262000F056
:109F500031F815218903084302460021262000F02C
:109F600068F900222621362000F058F900F036F872
:109F7000206000207CBD0000F40000203001CADE1B
:109F800000000020FFFD000038B5094C89B280B206
:109F90006B46022200F028F8002806D16846407877
:109FA000010268460078081884B2204638BD0000D7
:109FB000FFFF000038B50024E44389B280B26B464D
:109FC000042200F011F8002806D103216846435C02
:109FD0002202D418491EFAD5204638BD10B50021FA
:109FE0000846FFF7E7FF10BD38B5002909D0402427
:109FF00020436C462070C8B27F2906D860700220CA
:10A000000AE069460870012006E0802420436C467F
:10A010006070C809A0700320694600F0A5FA38BD39
:10A0200010B5144603460A4621461120FFF7DCFF0F
:10A0300010BD10B50346052200211520FFF7D4FFFF
:10A0400010BD10B50346052200211720FFF7CCFFF5
:10A0500010BD38B5054600206946087000F0C4F808
:10A06000FF2401342246002D01D0032212020021D8
:10A070000D2000F0D3F8002D13D06B4601220321F0
:10A080000F20FFF7B1FF68460078000709D5FFF7FA
:10A09000AFFE224600210D2000F0C0F80020C04392
:10A0A00038BD002038BD10B5024601210A2000F05D
:10A0B000C0F810BD10B5044600211A20FFF77AFF42
:10A0C000000D22030005120B024300211A2000F0AC
:10A0D000B0F810BD10B5024602492E2000F09EF8DF
:10A0E00010BD000004180000F8B505466B460122BB
:10A0F00003210420FFF778FF0126114C3607002DBD
:10A100000DD02A4600210C2000F088F86946087816
:10A110001021084369460870A069304307E069468A
:10A120000878EF21084069460870A069B0430B46E3
:10A13000A06101220321042000F08AF8F8BD00008C
:10A14000F400002010B502460021182000F066F847
:10A1500010BD0000F8B50746002568460570B80731
:10A16000204C2E4600280ADA8020694608706B468B
:10A17000012200210D2000F06BF801202073F80768
:10A180006946087821D006210843694608706B4665
:10A19000012200210D2000F05BF803210F20FFF7C2
:10A1A000F3FE8121C900084219D040206946087099
:10A1B0006B46012200210D2000F04AF80020FFF735
:10A1C00003FE00252673ED4309E00221084369469A
:10A1D00008706B46012200210D2000F039F8284656
:10A1E000F8BD0000140100201CB56B4601220321BC
:10A1F0000F20FFF7F9FE684600784022C1091040A1
:10A20000C9014000814208D0012069460871024618
:10A2100001AB03210D2000F01BF81CBD08B56B46F7
:10A220001A70120A5A7089B280B2022200F010F835
:10A2300008BD38B500236C46E254120A5B1C042B9F
:10A24000FADB89B280B22346042200F001F838BD5F
:10A2500038B58024002909D0C02528436D462870D0
:10A26000C8B27F2907D86870022009E020436946F8
:10A270000870012004E020436870C809A87003201A
:10A28000694600F0ADF938BD10B514460123121827
:10A290009B029A4202D90020C04310BD0B46821E89
:10A2A00021460920FFF7D4FF002010BD10B5054A54
:10A2B0008905126901430A4300210820FFF7B9FF0D
:10A2C000002010BDF400002038B504466B46012282
:10A2D0000E212B20FFF788FE68460078E106400932
:10A2E0004001C90E0143684601706B4601220E21F0
:10A2F0002B20FFF7ADFF38BD10B5002142541C06DE
:10A30000120A22431B0A491C0429F7DB10BD000076
:10A3100013B501231A4669460248FDF743FB00982E
:10A320001CBD0000101500207CB5002425466846A1
:10A33000FFF77FFE04206946220E2D0215432202FC
:10A340000C5C1443401EF7D5204629467CBD7CB5E5
:10A35000002425466846FFF774FE04206946220E55
:10A360002D02154322020C5C1443401EF7D52046F3
:10A3700029467CBDFCF7FCFAFEF73CFDFDF77CFEB0
:10A3800037493848002522C005608561C5613649D6
:10A390000562C1600838FCF705FCFDF759FEFDF7C2
:10A3A0003BFFFDF717FFFDF71FFE052601223607CD
:10A3B000D1033046FCF7C7FAFEF7E4FBFDF718FDC2
:10A3C000FBF798FBFBF766FB0721B015FFF7E4FCF2
:10A3D000264C0A21208A012248436083170339460C
:10A3E0003046FCF7B0FA1F48C82221498830FDF7F3
:10A3F0007BFA204EE07800282FD0FEF7FBFCE570BA
:10A40000FBF78EFD20700F2809D90122394630460E
:10A41000FCF799FAFEF764FD0022394609E00122B3
:10A4200051033046FCF78FFAFEF75AFD0022012156
:10A4300049033046FCF787FAFDF71EFC608B0028C5
:10A4400001D0401E60830C48618B00780843D1D155
:10A4500001210846FCF798FCCCE7FDF70DFCC9E7A5
:10A46000007C004088140020FFFF0000BC0000209A
:10A47000580C0020000400503600002010B586B0B3
:10A480001748FCF714FB14216846FAF790FE1548AC
:10A4900000900320019000200290052069460007EB
:10A4A000FCF78CF969461048FCF788F969460F48B3
:10A4B000FCF784F901210846FCF766FCFF2401340F
:10A4C0002046FCF739FC0A4908680422104308605A
:10A4D0002046FCF741FCFCF747FC06B010BD00002D
:10A4E00088140020FFFF0000000400500008005006
:10A4F0000070004010B50122920218491848FBF77D
:10A500006FFB1648174902888A4225D00180042132
:10A510008180FF21F531C1800A21018100211E22A5
:10A520004181D24382810122C28101840182418220
:10A530008182C182018381834323C38602230387EF
:10A54000782343878287C287024640321184518430
:10A550009184C18300F02EF810BD0000200D002072
:10A5600000FC0008AA550000F0B58C460025102616
:10A57000052109078E620E4C08E067467F5DE760A3
:10A58000A768FF07FCD0E7681F706D1C8542F4DBED
:10A590000020074606E0E760A568ED07FCD0E56807
:10A5A0001D54401C9042F6D38E610020F0BD000087
:10A5B0000030014070B572B60124074DA402214657
:10A5C0002846FBF7F3FA002804D022460349284620
:10A5D000FBF790FB62B670BD00FC0008200D002068
:10A5E000F0B50025102605279C463F070B46BE62A6
:10A5F0000C4C06E0595DE160A168C907FCD0E16838
:10A600006D1C8542F6DB002007E06146095CE160D5
:10A61000A168C907FCD0E168401C9042F5D3BE6137
:10A620000020F0BD003001400000010203040005DD
:10A63000405C0000A05C0400C06C0800805C04006A
:10A64000E03F1E00E07D1E0007A9022570889B8860
:10A650000A001600010006000100020087008D00BC
:10A660002D001A3152001A339A001A351D011A377B
:10A670006B003B31BE003B335E013B3596023B37FE
:10A68000000099599959EB518F421E45142E0080B4
:10A69000EB51F5283333E13A703DE13AC235852B71
:10A6A000C2353333C235C235AE47E13A5138A330F3
:10A6B00051380000000000000000010203040607FA
:10A6C0000809030406080C101820300000000001DF
:10A6D00002030400F4A6000800000020F4000000BB
:10A6E00028970008E8A70008F4000020441900009B
:10A6F0003897000800070400091E080540082609CD
:10A700001040085608054008261D040008BE1D0418
:10A710000008BED8BC401008010000000000C8427C
:10A720000000000000000000000000000000000029
:10A730000000000000000000000000000000000019
:10A740000000000000000000000000000000000009
:10A750008C0A000000000000000000000000000063
:10A7600000000000000000000000000000000000E9
:10A7700000000000000000000000000000000000D9
:10A7800000000000000000000000000000000000C9
:10A7900000000000000000000000000002020400B1
:10A7A0000909010200810000000000000100000012
:10A7B0000000000000000000000000000000000099
:10A7C0000000000000000000000000000000000089
:10A7D0000000000000000000000000000000000079
:08A7E000000020000000000051
:04000005080050C1DE
:00000001FF
